:020000004A2C88
:08000800FF00030E8312031335
:10001000A0000A0EA100040EA2008A110A126F2C81
:1000200000000000D00B10280800C308031D192889
:100030000800F9300000000000000000000000008F
:1000400000000000000000000000000000000000B0
:1000500000000000FF3E031D1A2800000000000001
:100060000000000000000000000000000000000090
:10007000000000000000000000000000C30B192871
:100080000800FA30C3001520FA30C3001520FA30FA
:10009000C3001520FA30C3001520C20B4128080008
:1000A0000130D1005008FF3903195A280310D10D2F
:1000B000FF3E5328FF305106D10006058600080098
:1000C0000130D1005008FF3903196A280310D10DFF
:1000D000FF3E63285108060486000800FA308312A8
:1000E0000313D000102008000130D00050206E20F3
:1000F000CF1F7E280730D000602081280730D00035
:1001000050204F1F87280630D00060208A280630F4
:10011000D0005020CF1E90280530D00060209328BA
:100120000530D00050204F1E99280430D0006020A8
:100130009C280430D00050206E200230D000602077
:100140006E200230D00050206E20CF0EF030CF0550
:10015000CF1FAE280730D0006020B1280730D00074
:1001600050204F1FB7280630D0006020BA28063034
:10017000D0005020CF1EC0280530D0006020C328FA
:100180000530D00050204F1EC9280430D000602018
:10019000CC280430D00050206E200230D0006020E7
:1001A0006E200230D000502008000130D0005020D6
:1001B0006E20C21FDF280730D0006020E228073001
:1001C000D0005020421FE8280630D0006020EB28E5
:1001D0000630D0005020C21EF1280530D00060202B
:1001E000F4280530D0005020421EFA280430D000F8
:1001F0006020FD280430D00050206E200230D00056
:1002000060206E200230D0005020080083120313BB
:10021000D00150206E20080083120313D00160200B
:100220006E20080006214208CF0074200C214203F2
:10023000031D08000A30C30015200800C901CC01C5
:10024000CD014708CA00CB01C9190800481C2E2956
:100250004A08CC070318CD0A4B08CD07C80C031079
:10026000CA0DCB0DC90A2429CB01CE01CF01470805
:10027000CC004808CD004B1A0800491C45294C0801
:10028000CE074D0803184D0FCF070310CA0CC90C39
:100290000310CC0DCD0DCB0A3B29CB01CC01CE01F7
:1002A000CF01CD014D1A08000310CE0DCF0DC70DA3
:1002B000C80DCB0DCC0D4A084C02031D612949081D
:1002C0004B02031C6A294908CB024A08031CCC03D1
:1002D000CC024E14CD0A5229643083120313C3009A
:1002E00015208316860102308312D000502006218B
:1002F0003830C200D5200530C30015203830C20088
:10030000D5200230C30015203830C200D52002307D
:10031000C30015202830C200D5200230C3001520AC
:100320002830CF0074200230C30015200830CF00E1
:1003300074200230C30015200C30CF00742002302E
:10034000C30015200630CF0074200230C3001520F2
:100350008030CF0074200230C30015200C2108002B
:10036000420803178D0083168C130C1483120C089B
:100370000313C30008000C21CD0183134318831716
:1003800042084D0784000008CE004E08403A031989
:100390000800CE08031908004E08CF007420CD0ACB
:1003A00083134318831742084D0784000008CE00CA
:1003B000CE08031DC52908000C21C501C60142084D
:1003C000C7004308C8001030C9002730CA004D21BB
:1003D0004E08C400C40803190C2A30304407CF006B
:1003E00074204408C700C8011030C9002730CA0073
:1003F00034214E08C5004F08C60045084202C70018
:10040000460A031846084302C8004708C2004808C5
:10041000C3006330C500C6014208C7004308C800D6
:10042000E830C9000330CA004D214E08C400C4089A
:10043000031D202A6330450603194608031D3F2A81
:1004400030304407CF0074204408C700C801E830AA
:10045000C9000330CA0034214E08C5004F08C60049
:1004600045084202C700460A031846084302C8006E
:100470004708C2004808C3006330C500C6014208EF
:10048000C7004308C8006430C900CA014D214E08A6
:10049000C400C408031D522A6330450603194608E8
:1004A000031D6E2A30304407CF0074204408C70073
:1004B0006430C8001E214C08C5004D08C600450820
:1004C0004202C700460A031846084302C80047080C
:1004D000C2004808C3006330C500C6014208C70017
:1004E0004308C8000A30C900CA014D214E08C400A3
:1004F000C408031D812A6330450603194608031DFD
:100500009A2A30304407CF0074204408C7000A30CC
:10051000C8001E214C08C5004D08C600450842020F
:10052000C700460A031846084302C8004708C2002D
:100530004808C30030304207CF00742008008312FF
:10054000031385018601870188018901FF30831625
:1005500085008601FD308700FF3088008901831205
:10056000360881008430831681006C2105309700A5
:100570008C018D018B160B1783160C158B170F3002
:100580009F00051483129F171F130130AF00043022
:100590009200FF308316920083129B010C309D0065
:1005A000080006214303031DDB2A4208803EC400E5
:1005B0004403CF0074204308023A031DE82A42088E
:1005C000803EC40040304407C4004403CF00742080
:1005D0000C210800013083120313C200122108000D
:1005E000AF08031DF62A6330C30008002F03031D64
:1005F0000A2B1F149F111F129F124208C400C40D22
:10060000C40D440DF839C2001F049F002E08AD0030
:100610000230AF002F08023A031D172BAD08031D4F
:10062000132B0330AF002D08003C031CAD032F0833
:10063000033A031D1E2B1F150430AF002F08043A88
:10064000031D2F2B1F192F2B83161E088312AB009F
:100650001E08AC001F100130AF00C3000800C3012A
:1006600008009F22C201B0214308BD000130C20032
:10067000B0214308BE00C2013E08A60042083D0763
:10068000A5000318A60AEA225730C4006930C50045
:100690006330C6006B30C7006530C8006C30C900DD
:1006A0006D30CA006130CB00CC010030CD00443049
:1006B000C2004D08C300BB210130C2000230C3009C
:1006C000D1227330C4006330C5006830C600693081
:1006D000C7006E30C8006530C900CA010030CB00C9
:1006E0004430C2004B08C300BB210130C20041208E
:1006F000EA222830C4006330C5002930C60020300B
:10070000C7004830C8006530C9006C30CA006D3081
:10071000CB00CC010030CD004430C2004D08C300F6
:10072000BB210130C2000230C300D1227530C400A9
:100730007430C5002030C6005730C7006530C8008F
:100740006930C9006730CA006C30CB00CC01003082
:10075000CD004430C2004D08C300BB210130C200AF
:100760004120EA220130C2000230C300D1222030F1
:10077000C400C5010030C6004430C2004608C300B2
:10078000BB210A30C2000230C300D1223F03031D47
:10079000D42B7630C400C5010030C6004430C200FE
:1007A0004608C300BB21DE2B7230C400C5010030F7
:1007B000C6004430C2004608C300BB210130C2005D
:1007C000C300D1222030C400C500C600C700C80045
:1007D000C9010030CA004430C2004A08C300BB212E
:1007E0000130C200C300D1222708C2002808C3007C
:1007F000DC212708A9002808AA00C201F02243032F
:10080000031D062C2C08BB003B089B00290827066B
:10081000031D0E2C2A0828060319FD2B0130C200E7
:10082000C300D1222030C400C500C600C700C801E3
:100830000030C9004430C2004908C300BB21013068
:10084000C200C300D1222708C2002808C300DC214F
:100850002708A9002808AA000A30C2000230C300F5
:10086000D1223F03031D3F2C7630C400C501003068
:10087000C6004430C2004608C300BB21FD2B7230C5
:10088000C400C5010030C6004430C2004608C300A1
:10089000BB21FD2B83120313AF01AD010F30AE005E
:1008A000B001B101B201B301B401B501BF30B6006E
:1008B000B701B8010130B900BA01BB010130BC0079
:1008C0000130A300A401A701A8010130A900AA01D9
:1008D0000130BF00C001C1018A110A12312B0B1D6A
:1008E000AF2C8312031336088100B00A30080A3A8D
:1008F000031D832C3108003C031CB1033508003C68
:10090000031CB503B0013008053A031DAE2CFF30BF
:100910000806B2003F303205B200B2080319992C24
:10092000B308031D992C0A30B1000130B30032081E
:10093000B400B208031DA62C3303031DA62CB10876
:10094000031DA62C0A30B1000230B3003308023A6E
:10095000031DAE2CB108031DAE2CB3010B11831285
:1009600003130C1DF72C071CB82C0130BF00B92C49
:10097000BF013F03031DD92CA30A031DC02CA40AE9
:1009800024082602031DC62C230825020318F62C72
:100990000130A300A401A70A0319A80A2808273CCC
:1009A000031DD42C27080F3C0318F62CA701A8011F
:1009B000F62CA3080319A403A303A308031DF62C14
:1009C000A408031DF62C2508A3002608A400A708E8
:1009D000031DF22CA808031DF22C0F30A7002730AE
:1009E000A800F62CA7080319A803A7030C11220ED0
:1009F0008400210E8A00200E8300FF0E7F0E090066
:00000001FF
